:100000000000000000000528090007309F0083164B
:100010009F01EB3086008A018312752882008207D7
:10002000033443346C346B348207063443346F3406
:100030006D346D346F346E34820703344434693464
:1000400072348207043444346F346E34653482076A
:1000500004344634613469346C34820703344634E2
:100060002F34533482070B344D346F3474346F346F
:10007000723432345F3454346534733474348207E8
:1000800004344D346F3464346534820703344D34A2
:100090002F344434820705344D346F3474346F3454
:1000A0007234820705340034013410348034FF3454
:1000B00082070434523461346D347034820706345C
:1000C0005334633461346C346534723482070634DB
:1000D0001034203440348034FF3400348207053437
:1000E00053347034653465346434B6233330DB0004
:1000F0005924B623A8010616C8234A08A5006C2473
:100100006C2430302502031C95283A302502031850
:1001100095282508DA005324280DA900A90D290DDA
:10012000F8392507D03EA8000C2973302502031D9D
:10013000A2282508DA005324B6232808D1000D246C
:10014000A8010C2977302502031DCE282508DA00E6
:100150005324B6232808D1000D24A801A701053097
:1001600027020318BE28E7234D08A90020302707DF
:100170008400290883138000A70AAF28A70105304F
:1001800027020318CC282030270784008313000897
:10019000CB00CE23A70ABF28B6230C29693025023D
:1001A000031DDF282508DA005324B623FD30D100D3
:1001B0000D24ED23ED23ED23FE23FE230C297430C3
:1001C0002502031DEC282508DA005324B62328084D
:1001D000B3009C21A8010C2963302502031DF928D6
:1001E0002508DA005324B6232808AA000D21A80107
:1001F0000C29FC30250203190C293C30DA00532469
:100200002508CB00CE233E30DA005324B62328083D
:10021000CB00CE23B623A8017B283B30B2002A08AE
:100220003202B1000230AC00FF30AD00F030AE0061
:100230005430DA0053240530CB00CE233108CB00F4
:10024000CE23B6234330DA005324FA30D1000D24F4
:10025000E7234D08CB00CE23FB30D1000D24B001A5
:10026000AF01861A31293429861A3A29B00A0319AE
:10027000AF0A34294830DA0053242F08CB00CE23AC
:100280004C30DA0053243008CB00CE2306302F0246
:1002900003186F2905302F02031C6A293008310228
:1002A000031C622931083002031C5A29AB01AD013D
:1002B000AE016129F830AB003108B20030083202DB
:1002C000AD006929F930AB003008B20031083202C4
:1002D000AD006E29F830AB003108AD007629F93059
:1002E000AB00FF30B20031083202AD004530DA0019
:1002F00053242D08CB00CE234D30DA0053242E0892
:10030000CB00CE232D082E02031D8929B6230034ED
:1003100097292E082D02031C9429AC03031D932951
:10032000AE0A0230AC0097292D08AE00AD0A2B08AA
:10033000D1000D24B62322293308031DA129FF3043
:10034000B30001303305031D1923A830D1000D245B
:10035000023033050319CC295F30DB005924B62362
:10036000BA0108303A020318CC2990303A04D1007F
:100370000D249930D1000D24E7234D08BF003A0227
:100380000319CA293F08CB00CE235F30C8003030A4
:10039000C900BD23BA0AB1299530D1000D2404301B
:1003A000330503190D2A2E30DB005924B623823081
:1003B000D1000D24FF30D1000D243C30D1000D249C
:1003C000FF30B70037080319EC29A130D1000D2404
:1003D000E7234D08B700E229A030D1000D24E72320
:1003E0004D08BF003F030319FD293F08CB00CE2372
:1003F0002E30C8003730C900BD23A030D1000D24F5
:10040000E7234D08BF0003190D2A3F08CB00CE2378
:100410002E30C8003830C900BD23A830D1000D24CB
:10042000083033050319112BBC0105303C020318B9
:10043000112B3C0A8A015120BB00B801023038025E
:1004400003180F2BB6010230360203180D2BB90129
:100450000230390203180B2B5930DB0059243B08BA
:10046000CB00CE234030DB0059243808CB00CE230C
:100470001D30DB0059243608CB00CE234B30DB0087
:1004800059243908CB00CE23B6230310380D390484
:100490008838D1000D2480303904D1000D243B0868
:1004A000D1000D249E303904D1000D24E7234D08DE
:1004B000BF003B020319642A3F08CB00CE2359300A
:1004C000C8003130C900BD233B08031DD12ABE013D
:1004D000FF303E020318AC2A0310360D3904BF006A
:1004E0003E0E0F39C0000F303E05400203198D2A21
:1004F0000F303E05031D862A3E0CC000400C3F39DC
:100500003F04D1000D2440303F048C2A3E0DC00032
:10051000400D3C393F044038922A3E0CC000400C4C
:100520003C393F04D1000D249A303904D1000D2408
:10053000E7234D08BF003E083F020319AA2A3E08E0
:10054000CB00CE233F08CB00CE236F30C800323023
:10055000C900BD23BE0A682A3E080319D02A031029
:10056000360D39048438D1000D243E08D1000D2405
:100570009A303904D1000D24E7234D08BF003E080E
:100580003F020319CE2A3E08CB00CE233F08CB0002
:10059000CE236F30C8003330C900BD23BE03AC2A60
:1005A000092BBD0106303D020318092B3D0A8A01C3
:1005B0006620BE000310360D39048438D1000D24A6
:1005C0003E08D1000D243E03BF000830B400FF30C8
:1005D000B5003F083E020319F42AA2303904D100C5
:1005E0000D24E7234D08BF00B50BE92AB40BE72A19
:1005F0003F083E020319072B3F08CB00CE233E08DD
:10060000CB00CE235930C8003430C900BD23BD0A09
:10061000D22AB90A282AB60A232AB80A1E2ABC0AEC
:10062000152AA830D1000D242230DB005924B6232E
:100630000034FD30D1000D240130C300C030C400AF
:100640008F23C301C130C4008F230E30C300C230DA
:10065000C4008F230230C300C330C4008F23C30102
:10066000C430C4008F23C301C530C4008F23C3012D
:10067000C630C4008F23C301C730C4008F23B62304
:100680009A239A23A423A423AF234708FD30D10043
:100690000D240130C300C830C4008F23FE30D100C8
:1006A0000D24E7234D08C100FF30D1000D24FF3099
:1006B000D1000D24FE30D1000D24E7234D08C200E7
:1006C000023042020319692B1530C800C930C90035
:1006D000BD23FB30D1000D24E7234D080319752BF2
:1006E0001530C800CA30C900BD23FA30D1000D242E
:1006F000E7234D08C100F930D1000D24F830D100B6
:100700000D24FA30D1000D24E7234D0841020319CE
:100710008E2B1530C800CB30C900BD230034AF2369
:10072000470843020319992B1530C8004408C90033
:10073000BD2300340830C500AF234708CB00CE23CB
:10074000C50B9C2BB6230034AF234708C600AF234C
:100750004708DA005324C60BA72BB6230034FC301D
:10076000D1000D24E7234D08C70000340D30DA0016
:1007700053240A30DA00532400342830DB00592493
:100780004808DB0059244908CB00CE23B6230034A7
:100790000230D20013245308CA0000344B0ECC00A0
:1007A000CC0C4C0C0339303EDA0053244B0CCC00FB
:1007B000CC0C4C0C0739303EDA00532407304B0583
:1007C000303EDA0053242030DA0053240034203045
:1007D000D20013245308CD0000340830CE00F72394
:1007E0004F08CB00CE23CE0BEF2BB6230034FC30CA
:1007F000D1000D24E7234D08CF000034F7234F0824
:10080000D000CB00CE235008D000F7234F08DA00E9
:100810005324D00B052CB62300345108D6001030D9
:10082000D70038240034D401060852050319212CBE
:10083000D4035408031D1F2CFC30D30000346C2457
:10084000142C6C246C246C24D5010830D4006C2446
:100850000310D50C060852050319302C8030D5043E
:100860006C246C24D40B272C6C245508D300003442
:10087000FF305706D90086006C246C246C240830A5
:10088000D8005618FF30561C590886000310D60CA5
:100890006C246C246C24D80B412CFF3086006C2413
:1008A0006C246C2400345A08D6000430D700382455
:1008B0000034DD018A015B080E205D020318682CFC
:1008C0005D0A5B078A010E20DA005324DD0A5A2CE8
:1008D0002030DA00532400347230DE00DE0B6E2C40
:0208E0000034E2
:02400E00293F48
:00000001FF
